:100000000C9470000C948F000C948F000C948F0053
:100010000C948F000C9463050C948F000C948F004B
:100020000C948F000C948F000C948F000C948F0014
:100030000C94DD190C948F000C948F000C948F009D
:100040000C948F000C9438050C94431F0C948F0073
:100050000C948F000C9491000C948F000C948F00E2
:100060000C948F000C948F000C948F000C948F00D4
:100070000C948F000C948F000C948F000C948F00C4
:100080000C948F000C948F000C948F000C948F00B4
:100090000C948F004C22572262226D2278228322F8
:1000A0008E229922A422AF22BD22CB22D922E7227E
:1000B000F222FD220B23162321232C233723422354
:1000C0004D23582363236E23792384238F239A237C
:1000D000A523B023BF23CA23D523E023EB23F92391
:1000E00011241FBECFEFD0E1DEBFCDBF13E0A0E0F3
:1000F000B1E0E8E6F0E500E00BBF02C007900D922A
:10010000AE36B107D9F716E0AEE6B3E001C01D92F6
:10011000A83BB107E1F70E94A9000C9432280C9487
:1001200000001F920F920FB60F9211240F900FBE76
:100130000F901F901895AC0120E030E002C02F5FB7
:100140003F4FFA01E20FF31F80818823C1F7C901F5
:1001500008956F927F928F929F92AF92BF92CF92AB
:10016000DF92EF92FF920F93DF93CF9300D00F9225
:10017000CDB7DEB7F8940E94B30A0E942B108FEF20
:1001800084B915B881E0809378032F980E94240BDE
:1001900081E897E10E946F0B85E69CE00E94740B5A
:1001A00081E090E00E94790BDE011196E3EEF2E02F
:1001B00083E001900D928150E1F7CE0101960E94FB
:1001C000620F80E091E00E94001081E191E00E94C6
:1001D000F80F82E491E00E94F00F0E94380F4C016A
:1001E00068EC70E00E94870BC40160E070E00E9440
:1001F000AE0E3C01C401B30140E050E00E94AD0BE3
:10020000C401B30141E050E021E030E002E0A0E4AD
:10021000EA2EF12CCC24DD24F6EBAF2EF1E0BF2E3C
:100220000E94430EC401B30141E050E021E030E000
:10023000E4E5AE2EE4E0BE2E0E947B0E1092CD03CC
:100240001092CC031092CF031092CE030E94741B25
:100250008FE787B98AE288B90E948B0585E588B95E
:100260000E948B0518B80E94B1100E94B30A0E9428
:1002700030107894FFCF0F931F93CF93DF938C01AF
:1002800081349105F0F18091D8039091D903892BA5
:10029000C1F500D000D000D0EDB7FEB731968BE4A9
:1002A00091E0ADB7BEB712969C938E93119783E5FC
:1002B00091E09383828381EC90E0958384830E9414
:1002C0000D250F900F908AE591E0EDB7FEB7928370
:1002D0008183148303830E940D251092D50310920D
:1002E000D4031093D7030093D60381E090E090935A
:1002F000D9038093D80300E410E00F900F900F9083
:100300000F908BE268E00E94F50AC0E0D0E00DC0DB
:10031000E091D403F091D503EC0FFD1FE25EFA4F9C
:10032000608189E20E94F50A2196C017D10780F307
:100330008091CC039091CD03019749F48BE267E063
:100340000E94F50A1092CD031092CC030AC08BE2F2
:1003500063E00E94F50A81E090E09093CD038093E2
:10036000CC03DF91CF911F910F910895EF92FF92EF
:100370000F931F93CF93DF938091D8039091D9036C
:10038000019709F0B5C000D000D000D0EDB7FEB79E
:1003900031960BE411E0ADB7BEB712961C930E93E5
:1003A0001197B3E5EB2EB1E0FB2EF382E2828FEDE5
:1003B00090E0958384830E940D258DB79EB70696A5
:1003C0000FB6F8949EBF0FBE8DBF87E891E00E94E4
:1003D00022252091D4033091D5038091D6039091AA
:1003E000D7032817390708F083C000D000D000D009
:1003F000EDB7FEB73196ADB7BEB712961C930E930C
:100400001197F382E28282EE90E0958384830E94CA
:100410000D258DB79EB706960FB6F8949EBF0FBEFA
:100420008DBF84EA91E00E942225C091D603D0912D
:10043000D7038091D4039091D503C81BD90B809129
:10044000D4039091D503805C9F4F9093D503809304
:10045000D403C134D1052CF100D000D000D0EDB7C9
:10046000FEB73196ADB7BEB712961C930E93119797
:10047000F382E28288EE90E0958384830E940D25CA
:100480008DB79EB706960FB6F8949EBF0FBE8DBF70
:100490008CEC91E00E94222580E490E00E943B01D8
:1004A00027C000D000D000D0EDB7FEB73196ADB771
:1004B000BEB712961C930E931197F382E2828DEED3
:1004C00090E0958384830E940D258DB79EB7069694
:1004D0000FB6F8949EBF0FBE8DBF87EE91E00E94CD
:1004E0002225CE010E943B011092D9031092D8031D
:1004F000DF91CF911F910F91FF90EF900895CF92D0
:10050000DF92EF92FF921F93CF93DF93EC01109253
:10051000D5031092D4031092D9031092D80380917E
:10052000780381112F9A188112951F7000D000D086
:1005300000D0EDB7FEB731969BE4E92E91E0F92E9D
:10054000ADB7BEB71296FC92EE92119783E5C82E16
:1005500081E0D82ED382C2828BE690E0958384839B
:100560000E940D25EDB7FEB7319683EF91E0ADB750
:10057000BEB712969C938E93119712831382888133
:10058000848315820E940D258DB79EB706960FB6FF
:10059000F8949EBF0FBE8DBF143009F495C015307E
:1005A00058F4113029F11130A0F0123009F444C090
:1005B000133009F03DC164C0163009F4CDC01630C7
:1005C00008F4A6C0173009F4EBC0183009F030C1A8
:1005D0000BC18881863041F48A81813009F058C18D
:1005E000CE010E94AC1954C1CE010E94AA1050C184
:1005F00000D000D000D0EDB7FEB73196ADB7BEB792
:100600001296FC92EE921197D382C2828FE790E00D
:10061000958384830E940D258DB79EB706960FB6ED
:10062000F8949EBF0FBE8DBF83E192E00E94222509
:10063000CE010E9455132CC100D000D000D0EDB7E0
:10064000FEB73196ADB7BEB71296FC92EE921197F7
:10065000D382C28283E890E0958384830E940D2533
:100660008DB79EB706960FB6F8949EBF0FBE8DBF8E
:1006700085E292E00E942225CE010E94F51408C175
:1006800000D000D000D0EDB7FEB73196ADB7BEB701
:100690001296FC92EE921197D382C28287E890E084
:1006A000958384830E940D258DB79EB706960FB65D
:1006B000F8949EBF0FBE8DBF88E392E00E94222572
:1006C000CE010E942316E4C000D000D000D0EDB7C8
:1006D000FEB73196ADB7BEB71296FC92EE92119767
:1006E000D382C2828BE890E0958384830E940D259B
:1006F0008DB79EB706960FB6F8949EBF0FBE8DBFFE
:100700008BE492E00E942225CE010E94CE17C0C049
:1007100000D000D000D0EDB7FEB73196ADB7BEB770
:100720001296FC92EE921197D382C2828FE890E0EB
:10073000958384830E940D258DB79EB706960FB6CC
:10074000F8949EBF0FBE8DBF8EE592E00E942225D9
:10075000CE010E94FF1A9CC000D000D000D0EDB79F
:10076000FEB73196ADB7BEB71296FC92EE921197D6
:10077000D382C28283E990E0958384830E940D2511
:100780008DB79EB706960FB6F8949EBF0FBE8DBF6D
:1007900085E292E00E942225CE010E94740778C073
:1007A00000D000D000D0EDB7FEB73196ADB7BEB7E0
:1007B0001296FC92EE921197D382C28288E990E061
:1007C000958384830E940D258DB79EB706960FB63C
:1007D000F8949EBF0FBE8DBF81E792E00E94222554
:1007E000CE010E945C2054C000D000D000D0EDB7F4
:1007F000FEB73196ADB7BEB71296FC92EE92119746
:10080000D382C2828FE990E0958384830E940D2574
:100810008DB79EB706960FB6F8949EBF0FBE8DBFDC
:1008200084E892E00E942225CE010E94D02130C0AF
:1008300000D000D000D0EDB7FEB731968BE491E048
:10084000ADB7BEB712969C938E93119783E591E056
:100850009383828383EA90E0958384830E940D25AD
:100860008DB79EB706960FB6F8949EBF0FBE8DBF8C
:100870008AE992E00E942225888180931E0583E008
:1008800080931F051092200583E090E00E943B01B9
:100890008091780381112F98DF91CF911F91FF9064
:1008A000EF90DF90CF900895EF92FF920F931F93F8
:1008B000CF93DF93EC0100D000D000D0EDB7FEB7AE
:1008C00031960BE411E0ADB7BEB712961C930E93B0
:1008D000119723E5E22E21E0F22EF382E28287E3F4
:1008E00090E0958384830E940D250F900F90EDB7C3
:1008F000FEB7319686EA92E0ADB7BEB712969C93EA
:100900008E9311978981828313820E940D25809195
:10091000CE039091CF030F900F900F900F900197FF
:1009200009F04BC000D000D000D0EDB7FEB7319633
:10093000ADB7BEB712961C930E931197F382E28265
:100940008CE390E0958384830E940D258DB79EB73C
:1009500006960FB6F8949EBF0FBE8DBF8AEC92E04C
:100960000E94222520E030E0E091D003F091D103F5
:10097000E20FF31FDE01A20FB31F8C91E252FC4F76
:1009800080832F5F3F4F2034310571F78091D00372
:100990009091D103805C9F4F9093D1038093D003BB
:1009A0002091D0033091D1038091D2039091D30351
:1009B0002817390708F455C03FC000D000D000D038
:1009C000EDB7FEB73196ADB7BEB712961C930E9336
:1009D0001197F382E2828BE490E0958384830E94F6
:1009E0000D258DB79EB706960FB6F8949EBF0FBE25
:1009F0008DBF83ED92E00E9422251092D1031092C8
:100A0000D00320E030E0E091D003F091D103E20F79
:100A1000F31FDE01A20FB31F8C91E252FC4F8083C3
:100A20002F5F3F4F2034310571F73093D10320936E
:100A3000D0038981803448F41092CF031092CE0302
:100A40008EED93E00E947F020CC081E090E09093D5
:100A5000CF038093CE03898190E09093D30380935A
:100A6000D203DF91CF911F910F91FF90EF900895E6
:100A70001F920F920FB60F920BB60F9211242F9365
:100A80003F934F935F936F937F938F939F93AF9316
:100A9000BF93EF93FF930E947C108091770386BDF4
:100AA000FF91EF91BF91AF919F918F917F916F9146
:100AB0005F914F913F912F910F900BBE0F900FBE02
:100AC0000F901F9018951F920F920FB60F920BB6B2
:100AD0000F9211242F933F934F935F936F937F93C4
:100AE0008F939F93AF93BF93EF93FF930E94081050
:100AF000FF91EF91BF91AF919F918F917F916F91F6
:100B00005F914F913F912F910F900BBE0F900FBEB1
:100B10000F901F90189520E040E45CE9CA0101970E
:100B2000F1F72F5F2931D1F70895882321F0813023
:100B300061F084E008958EE08093A2038093A30384
:100B400088E18093C10081E008958EE0809387035F
:100B50008093880388E18093C90081E00895882309
:100B600021F0813081F084E008951092A203109268
:100B7000A3031092C5001092C4001092C1001092FD
:100B8000C20081E0089510928703109288031092AA
:100B9000CD001092CC001092C9001092CA0081E0E2
:100BA0000895882321F0813041F084E00895209356
:100BB000C5006093C40081E008952093CD00609348
:100BC000CC0081E00895623011F492E001C090E021
:100BD000882321F0813061F084E008958091C20083
:100BE000990F990F990F982B9093C20081E0089567
:100BF0008091CA00990F990F990F982B9093CA0072
:100C000081E00895663029F0673039F0653041F4AD
:100C100002C020E006C020E001C021E090E002C058
:100C200021E091E0882321F0813069F084E008958B
:100C30008091C200220F220F990F922B982B909334
:100C4000C20081E008958091CA00220F220F990FFF
:100C5000922B982B9093CA0081E00895653419F087
:100C60006F3419F405C021E001C020E090E002C01B
:100C700021E091E0882321F0813079F084E008952B
:100C80008091C2002295220F207E9295907F922B18
:100C9000982B9093C20081E008958091CA0022951C
:100CA000220F207E9295907F922B982B9093CA00D2
:100CB00081E00895982FFA018230B8F084E0089519
:100CC0002191992319F0913071F407C08091C000EF
:100CD00085FFFCCF2093C60006C08091C80085FF29
:100CE000FCCF2093CE00615070406115710541F733
:100CF00081E00895882321F0813051F084E0089547
:100D00008091C00085FFFCCF6093C60081E008950C
:100D10008091C80085FFFCCF6093CE0081E00895EC
:100D2000E82FDB01823010F084E008959A0116C0AC
:100D3000EE2321F0E13049F084E00DC08091C00045
:100D400087FFFCCF8091C60006C08091C80087FF56
:100D5000FCCF8091CE008D932150304012161306A7
:100D60003CF381E00895882321F0813049F084E04C
:100D700008958091C00087FFFCCF8091C600089540
:100D80008091C80087FFFCCF8091CE00089570E06D
:100D90000E945A0680931F051092200583E090E080
:100DA0000E943B0108950E94020680931F05109245
:100DB000200583E090E00E943B0108950E94020616
:100DC00080931F051092200583E090E00E943B0174
:100DD00008950E94E30580931F051092200583E08B
:100DE00090E00E943B0108950F930E94D1058093EB
:100DF0001F051092200583E090E00E943B010F91B7
:100E000008950E94AF0580931F051092200583E08E
:100E100090E00E943B010895882321F0813059F031
:100E200084E012C08EE08093A2038093A30388E144
:100E30008093C10008C08EE080938703809388036D
:100E400088E18093C90081E080931F0510922005FE
:100E500083E090E00E943B010895CF92DF92EF92F1
:100E6000FF920F931F93DF93CF93CDB7DEB78B0124
:100E7000CDB6DEB62DB73EB7261B370B0FB6F894AE
:100E80003EBF0FBE2DBFEDB6FEB60894E11CF11CAF
:100E9000B701A8010E94900680931F0520E030E072
:100EA0000AC0F701E20FF31F8081F901E05EFA4FFB
:100EB00080832F5F3F4F201731079CF3F801E05EDE
:100EC000FA4F1082C80103960E943B010FB6F894B6
:100ED000DEBE0FBECDBECF91DF911F910F91FF906F
:100EE000EF90DF90CF9008950F93FC018081809365
:100EF0001E058081843611F1853648F48236B1F0C2
:100F00008336E0F4803651F0813679F50BC08736B0
:100F100031F18836E9F0853641F515C082810E94AD
:100F20000C072CC082810E94010728C08281638146
:100F30004481258106810E94F40620C0828163815C
:100F40000E94E9061BC0828163810E94D30616C0FD
:100F5000828163813496AF010E94C7060FC063810E
:100F6000828170E00E942D0709C083E080931F05F5
:100F70001092200583E090E00E943B010F910895BC
:100F800087E28093860685E28093850690E29093BF
:100F900087061092880628E030E030938A06209376
:100FA000890683E28093920681E280939106909372
:100FB0009306109294063093960620939506089512
:100FC0000895089581E260919E060E94F50A0895B1
:100FD0008BE268E00E94F50A88E261E10E94F50A6E
:100FE0008FE268E00E94F50A8CE261E10E94F50A56
:100FF0008FE261E00E94F50A83E265E00E94F50A53
:1010000008950F931F938C0180E260E40E94F50A1B
:10101000F8016281605884E00E94F50AF80182813B
:1010200080939D061F910F9108950F931F93CF9367
:10103000DF93EC0128853985121613060CF03FC0AA
:101040008E819F81821793073CF583E268E00E94BE
:10105000F50A00E010E012C0EA85FB85E20FF31FFD
:1010600081E260810E94F50A8E819F8101969F83B3
:101070008E830F5F1F4F0830110539F02E813F819D
:1010800088859985281739073CF3288539858E810D
:101090009F818217930724F087E261E00E94F50A9E
:1010A0008B81813031F4898165E00E94F50A1B82D1
:1010B00006C0898161E00E94F50A81E08B83DF919F
:1010C000CF911F910F910895DF93CF9300D000D05F
:1010D000CDB7DEB7FC0132812381109298061092C1
:1010E000970681E080939406223031F12330B9F1E4
:1010F000213009F05FC080917106809399061092AB
:101100009A0681E796E090939C0680939B068681E1
:101110009781089721F480E490E097838683868105
:1011200097818034910509F045C088E090E0909364
:101130009A06809399063EC08681978190939A067D
:1011400080939906832F90E0880F991FE091830682
:10115000F0918406E80FF91F8081918127C0332325
:10116000B9F0832F90E0880F991FE091DC03F09194
:10117000DD03E80FF91F0190F081E02DF0939C064C
:10118000E0939B0680818093990610929A0612C084
:1011900094E099832A8389E08B839C8384E090E0A8
:1011A00090939A0680939906CE01019690939C069F
:1011B00080939B0681E996E00E9415080F900F909E
:1011C0000F900F90CF91DF910895CF93DF9382E23C
:1011D0000E94C10AC82F85FF1AC083E268E00E94FE
:1011E000F50AC6FF10C020919706309198068091AD
:1011F000990690919A06281739072CF481E996E010
:101200000E94150804C087E261E00E94F50ADF91A0
:10121000CF9108950F931F9388E00E94C10A082F71
:10122000182F86FF18C085E060E00E94F50A84E070
:1012300060E80E94F50A80E260E00E94F50A83E21D
:1012400068E00E94F50A87E261E00E94F50A85E005
:1012500062E00E94F50A14FF04C089E060EC0E947D
:10126000F50A07FF04C089E060ED0E94F50A1F91AE
:101270000F9108958AE00E94C10A80FF03C00E9476
:10128000E508089581FF0DC08AE20E94C10A80919D
:101290005E06813061F4E0916106F0916206099585
:1012A000089582E30E94C10A8AE30E94C10A089558
:1012B0008EE00E94C10A0895EF92FF920F931F9350
:1012C000DF93CF93CDB7DEB728970FB6F894DEBF84
:1012D0000FBECDBF86E20E94C10A86FF7FC08E018D
:1012E0000F5F1F4F49E0E42EF12CEC0EFD1E8091A4
:1012F00085060E94C10AF80181938F01EE15FF0552
:10130000B1F78E010F5F1F4F87E268E00E94F50A78
:1013100083E268E00E94F50A80E20E94C10A682F19
:101320006F7780E20E94F50A898190E08076907064
:101330008032910509F440C080349105D1F1892BA8
:10134000F1F5F80181818630D9F0873048F4813099
:10135000F1F18130C8F0833079F1853081F521C019
:10136000893019F18A3018F4883049F505C08A307F
:1013700071F18B3021F520C081E260919E0625C07D
:10138000C8010E94640823C083E268E00E94F50A55
:1013900081E261E00E94F50A81E260E00E94F50AC4
:1013A0000BC0C8010E94010812C0C8010E94E807D2
:1013B0000EC0C8010E94B10A83E265E006C080E267
:1013C0000E94C10A682F605880E20E94F50AF80165
:1013D00080818823D1F483E265E015C020919906CD
:1013E00030919A0680919506909196068217930700
:1013F00064F410929A061092990683E268E00E94C3
:10140000F50A87E261E00E94F50A28960FB6F89483
:10141000DEBF0FBECDBFCF91DF911F910F91FF9027
:10142000EF900895EF92FF920F931F93DF93CF9366
:10143000CDB7DEB7C054D0400FB6F894DEBF0FBEB4
:10144000CDBF8CE00E94C10A80FF03C00E945C09EE
:101450007AC081FF29C08EE20E94C10A8DE20E94FB
:10146000C10A89838E010F5F1F4F70E4E72EF12CB4
:10147000EC0EFD1E0F5F1F4F0E94E40AF8018083EF
:101480000E151F05B9F780916E03813039F4E09194
:101490007103F0917203CE01019609958FE268E025
:1014A0000E94F50A8FE22AC082FF2CC086E30E94C8
:1014B000C10A85E30E94C10A89838E010F5F1F4F15
:1014C00060E4E62EF12CEC0EFD1E0F5F1F4F0E9414
:1014D000E40AF80180830E151F05B9F780916F03A8
:1014E000813039F4E0917303F0917403CE010196D9
:1014F000099587E368E00E94F50A87E361E00E94AE
:10150000F50A21C083FF1FC08EE30E94C10A8E012D
:101510000F5F1F4F51E4E52EF12CEC0EFD1E8DE305
:101520000E94C10AF80181938F01EE15FF05B9F7FA
:1015300080917003813039F4E0917103F09172036E
:10154000CE0101960995C05CDF4F0FB6F894DEBF5F
:101550000FBECDBFCF91DF911F910F91FF90EF9004
:1015600008950895089581E080936A0080E18DBB1D
:1015700083B3876083BB84B3836084BB3F9A479AFD
:1015800008959FEF91B982B988B1805888B984B322
:1015900095E0892784BB88B1805888B984B38927AE
:1015A00084BB000011B888B1805888B984B322E0A8
:1015B000822784BB0000000080B198B1905898B990
:1015C00094B3922794BB089588B1805888B984B3A6
:1015D00022E0822784BB0000000080B198B19058BF
:1015E00098B994B3922794BB089582B98FEF81B9CB
:1015F00088B1805888B984B395E0892784BB88B1C5
:10160000805888B984B3892784BB62B988B180586F
:1016100088B984B391E0892784BB88B1805888B9A0
:1016200084B3892784BB089582B988B1805888B96A
:1016300084B391E0892784BB88B1805888B984B38A
:10164000892784BB0895089582E18093710681E023
:101650008093720680E191E0909374068093730604
:1016600010927506109276061092770688E08093A5
:10167000780610927A061092790610927C061092E3
:101680007B0610927E0610927D0610927F061092C5
:101690008006109281061092820610926E031092BC
:1016A0006F031092700310925E0610925F06109204
:1016B000600610926806109267061092DB03109283
:1016C000DA03089590937A068093790670937C06E6
:1016D00060937B0650937E0640937D060895909319
:1016E0007A0680937906089590937C0680937B0612
:1016F000089590937E0680937D06089580937506E5
:1017000008958093760608958093770608950F9341
:101710001F93CF93DF938C01CB01C0916706D091CB
:10172000680662E070E00E94D42710C09881298189
:101730008A81823041F4E92FF22F858190E0801771
:10174000910709F460870F80D885C02D209771F725
:10175000DF91CF911F910F9108959C01E091670651
:10176000F091680614C0A081B1818281843061F457
:10177000848190E08217930739F4868190E0861780
:10178000970711F413964C930780F085E02D30975E
:1017900051F708950895BF92CF92DF92EF92FF9292
:1017A0000F931F93CF93DF93EC01F62ED42EC22E0E
:1017B000B02EE0916706F0916806309799F489E0C1
:1017C00090E00E940B24FC019093680680936706CA
:1017D000D183C083F38210861782D282C4820583AC
:1017E000E6821AC0CF010780F085E02D3097D1F74F
:1017F0008C0189E090E00E940B24FC01D80118962E
:101800009C938E931797D183C083F382D282C48234
:10181000B582E68210861782DF91CF911F910F91DA
:10182000FF90EF90DF90CF90BF900895EF92FF92DE
:101830001F93CF93DF937C01C091DA03D091DB0338
:10184000209711F011E012C085E090E00E940B2477
:10185000FC019093DB038093DA03F182E082128231
:101860001482138210E012C01F5FEC018B819C81F7
:101870000097D1F785E090E00E940B24FC019C8347
:101880008B83F182E082128314821382812FDF9195
:10189000CF911F91FF90EF900895EF92FF920F93D9
:1018A0001F93CF93DF93E091DA03F091DB0380E0A5
:1018B00090E00380F481E02D01963097D1F7880FF6
:1018C000991F0E940B248093DC039093DD03C09149
:1018D000DA03D091DB0301C0EC01E880F9808A8152
:1018E00090E0880F991F0091DC031091DD03080F31
:1018F000191FF701808190E00E940B24F80180837A
:10190000918320E030E016C08A8190E0880F991F13
:10191000E091DC03F091DD03E80FF91F0190F08105
:10192000E02DE20FF31FD701A20FB31F8C9180832C
:101930002F5F3F4FF701808190E02817390724F38C
:101940008B819C81009741F6DF91CF911F910F9180
:10195000FF90EF9008956F927F928F929F92AF9237
:10196000BF92CF92DF92EF92FF920F931F93CF938C
:10197000DF93E0916706F0916806CC24DD2409C06E
:101980008281823019F40894C11CD11C0780F08533
:10199000E02D3097A9F7C601880F991F0E940B24EC
:1019A00080938306909384060894C108D108560159
:1019B000AA0CBB1C0894C11CD11CC1E0D0E0882437
:1019C00099244FC0E0916706F0916806A9E0EA2EDD
:1019D000F12C16C0A081B181848190E08C179D0705
:1019E00019F48381E80EF11C15968C9115978C17CC
:1019F00021F48281823009F44D010780F085E02DC9
:101A0000309741F700918306109184060A0D1B1D43
:101A1000C7010E940B24D8018C9311969C9320E05F
:101A200030E0E0918306F0918406EA0DFB1D019001
:101A3000F081E02DE20FF31FD401A20FB31F8C91B0
:101A400080832F5F3F4F2930310559F7E09183069E
:101A5000F0918406EA0DFB1D0190F081E02DE282F9
:101A60002196CC16DD060CF0ADCFE1E0EE2EF12C88
:101A700079E0A72EB12C6624772488249924A5C068
:101A8000A0916706B091680613C0ED91FC91119783
:101A90008181823049F4858190E08E159F0521F483
:101AA0008481682E772406C017960D90BC91A02DD6
:101AB000109759F701E010E07DC040916706509102
:101AC000680672C0DA01ED91FC9111978181843032
:101AD00009F065C016968C91169790E080179107D3
:101AE00009F05DC014968C9190E08E159F0509F069
:101AF00056C0DF019501BF01675F7F4FE09183060C
:101B0000F0918406E80DF91D0190F081E02DE20FBF
:101B1000F31F8D9180832F5F3F4FA617B70771F793
:101B2000E9E0F0E0AE0EBF1EA0916706B091680636
:101B300034C012968C911297853059F514968C9179
:101B4000149790E08E159F0521F515968C911597A9
:101B500090E080179107E9F4CD91DC911197950100
:101B6000BE01695F7F4FE0918306F0918406E80D26
:101B7000F91D0190F081E02DE20FF31F8991808320
:101B80002F5F3F4FC617D70771F787E090E0A80E89
:101B9000B91E17960D90BC91A02D109751F6DA0141
:101BA00017964D915C9118974115510509F08ACF10
:101BB0000F5F1F4F601671060CF07FCF0894E11C79
:101BC000F11CE2E0F0E08E0E9F1ECE14DF040CF05C
:101BD00057CFDF91CF911F910F91FF90EF90DF9042
:101BE000CF90BF90AF909F908F907F906F9008950F
:101BF000AF92BF92CF92EF92FF920F931F93CF932A
:101C0000DF93EC015B01122FE0916706F09168060B
:101C100018C0A081B181848190E0C817D90771F400
:101C2000868190E08A159B0549F48281843031F4E5
:101C300014968C9114978F5F14968C930780F0857F
:101C4000E02D309731F787E090E00E940B24FC01F3
:101C500087E0808385E0818312830383F582E482B9
:101C6000C682CF0167E045E02C2F0A2DEE240E94AA
:101C7000CB0BDF91CF911F910F91FF90EF90CF9001
:101C8000BF90AF900895AF92BF92CF92DF92EF9244
:101C9000FF920F93FC01A114B10401F142305105F0
:101CA00071F04330510599F041305105B9F481E0AC
:101CB00080935E06B0926206A09261060FC081E03A
:101CC00080935F06B0926406A092630607C081E02D
:101CD00080936006B0926606A092650620583F4F3A
:101CE000CF010E94F80D0F91FF90EF90DF90CF9001
:101CF000BF90AF900895AF92BF92CF92DF92EF92D4
:101D0000FF920F93FC014230510571F043305105B1
:101D100099F041305105B9F481E080936E03B0929F
:101D20007203A09271030FC081E080936F03B092A1
:101D30007403A092730307C081E080937003B09294
:101D40007603A0927503CF010E94F80D0F91FF90CA
:101D5000EF90DF90CF90BF90AF900895EF920F93E8
:101D6000CF93DF93082FE62EA0916706B091680607
:101D7000C0E0D0E014C0ED91FC91119785818017EF
:101D800051F412968C911297823029F484818F5FDE
:101D90008483C82FD0E017960D90BC91A02D10978A
:101DA00051F789E090E00E940B24FC0189E08083D8
:101DB00084E08183E2821382148215821682178264
:101DC0001086CF0169E044E0202F00E0EC2E0E9455
:101DD000CB0BCE01DF91CF910F91EF900895DF9261
:101DE000EF92FF920F931F93CF93DF93E82E162F5E
:101DF000F42ED22EA0916706B0916806C0E0D0E024
:101E000014C0ED91FC91119785818E1551F41296B5
:101E10008C911297823029F484818F5F8483C82F3C
:101E2000D0E017960D90BC91A02D109751F789E046
:101E300090E00E940B24FC0189E0808384E0818390
:101E4000128313821482F582D68207831086CF0113
:101E500069E044E02E2D00E0EC2E0E94CB0BCE0179
:101E6000DF91CF911F910F91FF90EF90DF90089538
:101E7000EF920F931F93109182061F5F10938206BB
:101E800089E090E00E940B24FC0189E0808389E0D6
:101E900090E09383828382E081831482158316828B
:101EA00080E887838AE18087CF0169E042E020E013
:101EB00000E0EE240E94CB0B812F90E01F910F9148
:101EC000EF9008950F931F93CF93DF938C01FC0144
:101ED00001900020E9F7E81BF90BCF01880F991F4B
:101EE0000E940B24EC01F80101900020E9F7E01BAF
:101EF000F10BEE0FFF1FE88323E02983AC0120E004
:101F000030E009C0F801E20FF31F8081FA018083FD
:101F100011822F5F3F4FF80101900020E9F73197C0
:101F2000E01BF10B4E5F5F4F2E173F0758F3CE01BA
:101F30000E94160C90E0DF91CF911F910F910895B0
:101F40000F931F93CF93DF938C01EB01CA010E9483
:101F5000620F282FE0916706F091680614C0A081F7
:101F6000B1818281843061F4848190E0801791078F
:101F700039F4868190E08C179D0711F418962C9304
:101F80000780F085E02D309751F7DF91CF911F91B9
:101F90000F910895CF93DF93EC01CB010E94620F64
:101FA000382FA0916706B091680615C09C911196D4
:101FB0002C91119712968C911297823041F4E92F4F
:101FC000F22F858190E08C179D0709F436831796D0
:101FD0000D90BC91A02D109749F7DF91CF910895F6
:101FE0000E94620F1816190614F480938106089552
:101FF0000E94620F1816190614F480938006089543
:102000000E94620F1816190614F480937F06089533
:102010001F93CF93DF9386E00E94C10AC82F86FFEB
:1020200002C00E94120AC2FF02C00E943A09C1FF08
:1020300002C00E940A0987E00E94C10A182F87E0A7
:1020400060E00E94F50A87E0612F0E94F50ADF91A7
:10205000CF911F91089581E062E00E94F50A0895F2
:102060000E94AB0C0E944D0C0E94C00780E061E012
:102070000E94F50A80E00E94C10A80FDFBCF81E04A
:1020800062E00E94F50A84E060E80E94F50A80E2BE
:1020900060E40E94F50A83E268E00E94F50A87E2A4
:1020A00069E00E94F50A8DE06FE00E94F50A8BE07E
:1020B0006FE00E94F50A89E068ED0E94F50A8FE062
:1020C00063E30E94F50A87E066ED0E94F50A85E069
:1020D00062E00E94F50A80E06CEC0E94F50A089527
:1020E0008EEC8093770381E080936E00809177037C
:1020F00086BD83E084BD08950895089583E08093AC
:102100001E0581E080931F058BE0809320052FE65C
:102110002093210593E69093220584E7809323057D
:10212000209324059093250581E6809326058EE66D
:10213000809327058FE58093280580E38093290508
:1021400081E380932A0510922B058EE090E00E9497
:102150003B010895FC018081833011F40E947E10C0
:1021600008951F9311E0812F0E944413812F60E096
:102170000E9447121F5F1431B1F718E1812F0E94AE
:102180004413812F60E00E9447121F5F1B32B1F79A
:102190001F910895FC0110827583648373836283A9
:1021A0004183478346830895FC019081818198177C
:1021B00010F080E00895A481B5816D9387818150EE
:1021C00019F48181A81BB1098783B583A4839FB7C4
:1021D000F89480818F5F80839FBF81E00895FC0128
:1021E00080818823E9F3A281B3812D91868181507A
:1021F00019F48181A81BB109B383A28386839FB799
:10220000F8948081815080839FBF822F0895FC01C4
:102210008081882319F42FEF3FEF13C0A281B3818F
:102220002D918681815019F48181A81BB109B38356
:10223000A28386839FB7F8948081815080839FBF5B
:1022400030E0C901089581E0089581E0089581E0BA
:10225000089581E00895FB011082833089F0843075
:1022600028F4813049F0823029F408C0843051F0DC
:10227000853051F085E0089583B107C086B105C06F
:1022800089B103C08CB101C08FB1808381E0089512
:10229000833089F0843028F4813049F0823029F489
:1022A00008C0843051F0853059F084E0089565B954
:1022B00005C068B903C06BB901C06EB981E008956B
:1022C00061BB81E00895882321F081E08093780349
:1022D0000895109278030895982F882321F081E0C3
:1022E0008093780302C0109278038BE180931E05DF
:1022F00090931F051092200583E090E00E943B011F
:10230000089598E190931E050E94481180931F053F
:102310001092200583E090E00E943B010895982FE1
:1023200089E180931E05933091F0943028F4913028
:1023300051F0923029F409C0943059F0953059F099
:1023400085E090E00AC093B107C096B105C099B18D
:1023500003C09CB101C09FB181E080931F059093A1
:1023600020051092210584E090E00E943B01089531
:1023700084E180931E0581E080931F051092200563
:1023800083E090E00E943B01089582E180931E0566
:1023900081E080931F051092200583E090E00E9469
:1023A0003B01089583E180931E0581E080931F0522
:1023B0001092200583E090E00E943B01089580E1A7
:1023C00080931E0581E080931F051092200583E015
:1023D00090E00E943B010895EF92FF921F93DF93DC
:1023E000CF93CDB7DEB727970FB6F894DEBF0FBEF9
:1023F000CDBF182F7B01BE016F5F7F4F0E94392236
:10240000882311F484E01BC0E12FF0E0E958FC4F71
:102410003281313011F086E012C0EB81FC81808185
:102420002F8190E002C0959587952A95E2F780FF6D
:1024300003C0F701308302C0F701108281E02796C4
:102440000FB6F894DEBF0FBECDBFCF91DF911F91C5
:10245000FF90EF900895DF93CF930F92CDB7DEB743
:102460009BE190931E05BE016F5F7F4F0E94EC11B0
:1024700080931F058981809320051092210584E0B7
:1024800090E00E943B010F90CF91DF9108950F9350
:102490001F93DF93CF93CDB7DEB727970FB6F8948E
:1024A000DEBF0FBECDBF182F062FBE016F5F7F4F5F
:1024B0000E943922882311F484E025C0E12FF0E046
:1024C000E958FC4F8281823011F086E01CC0E9811E
:1024D000FA81002359F080819F8121E030E002C021
:1024E000220F331F9A95E2F7822B0BC030812F8188
:1024F00081E090E002C0880F991F2A95E2F780954D
:102500008323808381E027960FB6F894DEBF0FBE49
:10251000CDBFCF91DF911F910F9108959AE19093D4
:102520001E050E94471280931F051092200583E02C
:1025300090E00E943B0108951F93DF93CF93CDB7A6
:10254000DEB727970FB6F894DEBF0FBECDBF182FAA
:10255000BE016F5F7F4F0E943922882311F484E00F
:1025600015C0E12FF0E0E958FC4F81E08283ED8156
:10257000FE8130812F8181E090E002C0880F991F99
:102580002A95E2F780958323808381E027960FB612
:10259000F894DEBF0FBECDBFCF91DF911F9108959C
:1025A00095E190931E050E949C1280931F05109246
:1025B000200583E090E00E943B0108951F93DF9384
:1025C000CF93CDB7DEB727970FB6F894DEBF0FBE17
:1025D000CDBF182FBE016F5F7F4F0E943922882325
:1025E00011F484E014C0E12FF0E0E958FC4F82E0E0
:1025F0008283ED81FE8120813F8181E090E002C0F5
:10260000880F991F3A95E2F7282B208381E02796BF
:102610000FB6F894DEBF0FBECDBFCF91DF911F91F3
:10262000089596E190931E050E94DE1280931F0587
:102630001092200583E090E00E943B0108951F93D3
:10264000182F0E94DE12813071F4812F61E00E9408
:102650004712813041F4E12FF0E0E958FC4F83E06C
:10266000828381E001C084E01F91089597E19093F7
:102670001E050E941F1380931F051092200583E002
:1026800090E00E943B0108950E94DE12089591E1BE
:1026900090931E050E94DE1280931F051092200564
:1026A00083E090E00E943B010895FC018081863127
:1026B000E9F1873178F4823131F1833130F48031BE
:1026C000D1F0813109F050C01AC0843131F1853127
:1026D00048F51EC08931B9F18A3130F4873151F1A2
:1026E000883109F041C02AC08B31B1F18B3178F1CA
:1026F0008C31D1F535C082810E94DF11089582812D
:102700000E9447130895828163810E94C511089534
:10271000828163810E94D2110895828163810E9427
:10272000B811089582810E94D012089582810E947A
:102730001113089582810E94361308958281638166
:102740000E948111089582810E948F1108958281D3
:1027500063810E948E12089582810E942B12089537
:1027600082810E946C11089580931E0583E08093FE
:102770001F051092200583E090E00E943B01089520
:10278000E82F8A50883018F024E030E00CC0F0E0E8
:10279000E958FC4F84E0828380917C00806C8093B8
:1027A0007C0021E030E0C9010895E82FF0E0E9580D
:1027B000FC4F8281843019F024E030E003C01282A3
:1027C00021E030E0C901089510927C00823039F098
:1027D000833049F0813061F022E030E00BC080911D
:1027E0007C00806403C080917C00806C80937C00BE
:1027F00021E030E0C901089593E890937A00909128
:102800007C00907F982B90937C0080917A0080646C
:1028100080937A0080917A0086FDFCCF80917800C9
:102820009091790040E050E020E030E080917A0023
:10283000806480937A0080917A0086FDFCCF80913D
:10284000780090917900280F391F4F5F5F4F443017
:10285000510561F780917A008F7780937A003695E1
:10286000279536952795C9010895982F83E280937F
:102870001E0510927C00923039F0933049F091306F
:1028800061F082E090E00BC080917C00806403C026
:1028900080917C00806C80937C0081E090E080934C
:1028A0001F051092200583E090E00E943B010895EF
:1028B00091E290931E05E82FF0E0E958FC4F8281E9
:1028C000843019F084E090E003C0128281E090E04F
:1028D00080931F051092200583E090E00E943B0149
:1028E0000895E82F80E280931E058E2F8A5088304D
:1028F00018F084E090E00CC0F0E0E958FC4F84E070
:10290000828380917C00806C80937C0081E090E0E9
:1029100080931F051092200583E090E00E943B0108
:102920000895CF93DF93982FEB0119821882E82F37
:10293000F0E0E958FC4F8281843019F026E030E065
:1029400032C081E1891B0E94FC139983888300D0E7
:1029500000D000D0EDB7FEB7319686EE92E0ADB76D
:10296000BEB712969C938E9311978EEE92E093834E
:1029700082838BE890E0958384830E940D250F90DD
:102980000F9084EF92E0EDB7FEB792838183888148
:102990009981948383830E940D2521E030E00F907C
:1029A0000F900F900F90C901DF91CF910895DF93A1
:1029B000CF9300D0CDB7DEB792E290931E05BE0153
:1029C0006F5F7F4F0E94911480931F0599818A81C8
:1029D000809320059093210584E090E00E943B01C4
:1029E0000F900F90CF91DF910895FC01808181328B
:1029F00071F0823218F48032B1F405C0823259F09D
:102A0000833289F40CC082810E94711408958281FE
:102A10000E945814089582810E94D71408958281DB
:102A20000E943514089580931E0583E080931F054E
:102A30001092200583E090E00E943B010895ECEBAA
:102A4000F0E08081846080838BE0809385038CE05C
:102A50008093860381E090E00895ECEBF0E08081C4
:102A60008B7F8083109285031092860381E090E033
:102A700008958093B800E9EBF0E080818C7F80833B
:102A80008081808381E090E008958091B900887F03
:102A900008958091B90084EA8093BC008091BC00C5
:102AA00087FFFCCF81E090E0089584E98093BC002B
:102AB0008091BC0084FDFCCF81E090E00895AC01E2
:102AC00020E030E094E80EC0FA01E20FF31F8081AD
:102AD0008093BB009093BC008091BC0087FFFCCF2B
:102AE0002F5F3F4F261737077CF3089584E88093C4
:102AF000BC008091BC0087FFFCCF8091BB00089593
:102B000085E380931E0581E080931F0520E030E07F
:102B100094E80EC09093BC008091BC0087FFFCCF6E
:102B20008091BB00F901E05EFA4F80832F5F3F4F39
:102B3000261737077CF3FB01E05EFA4F1082CB01CA
:102B400003960E943B010895AC0120E030E094E838
:102B50000EC0FB01E20FF31F80818093BB009093B6
:102B6000BC008091BC0087FFFCCF2F5F3F4F241734
:102B700035077CF381E080931F051092200583E0E8
:102B800090E00E943B01089584E98093BC0080910D
:102B9000BC0084FDFCCF81E080931F0510922005CE
:102BA00083E090E00E943B0108958091B90084EA9F
:102BB0008093BC008091BC0087FFFCCF81E08093B4
:102BC0001F051092200583E090E00E943B010895CC
:102BD0008093B800E9EBF0E080818C7F8083808176
:102BE000808381E080931F051092200583E090E0B0
:102BF0000E943B010895ECEBF0E080818B7F8083A5
:102C0000109285031092860381E080931F05109235
:102C1000200583E090E00E943B010895ECEBF0E09A
:102C20008081846080838BE0809385038CE0809337
:102C3000860381E080931F051092200583E090E0D9
:102C40000E943B010895FC01808180931E058081D4
:102C50008433D1F0853338F4813379F0823381F0D5
:102C6000803331F507C08633E9F08633A0F087332F
:102C7000F9F41BC00E940E1608950E94FB150895DA
:102C800082810E94E8150895828190E03396BF0109
:102C90000E94A41508956381828190E070E00E94F3
:102CA000801508950E94D51508950E94C4150895B1
:102CB00083E080931F051092200583E090E00E943E
:102CC0003B010895782F613041F0613040F062306F
:102CD00041F0633009F059C007C060E006C060E011
:102CE00001C061E050E002C061E051E04330B9F062
:102CF000443028F4413059F0423078F40AC045306D
:102D000099F0453070F0463009F03FC010C021E026
:102D10000CC021E041E030E00DC021E009C020E01E
:102D2000F9CF20E041E005C020E040E0F4CF20E012
:102D300040E031E0239884B1866084B985B1817F19
:102D400085B980E090E0772311F081E090E075E0B4
:102D5000880F991F7A95E1F78065660F660F660FF9
:102D6000682B550F550F562B542B220F252B2CBD9E
:102D70003DBD88E080937E038AE080937F0389E0F5
:102D80008093800321E030E002C022E030E0C901FE
:102D900008951CBC1DBC10927E0310927F031092FC
:102DA000800381E090E00895AC0120E008C0E60FC8
:102DB000F71F80818EBD0DB407FEFDCF2F5FE22F80
:102DC000F0E0E417F5079CF381E090E00895DC0162
:102DD00020E030E040E050E014C01EBC08C083E0BA
:102DE000493E580714F088E008954F5F5F4F0DB4D7
:102DF00007FEF5CF8EB5FB01E20FF31F80832F5F37
:102E00003F4F2A173B074CF381E00895CF93DF93A0
:102E1000EC0120E030E0A0E0B0E018C0FE01E20FDD
:102E2000F31F80818EBD08C0119683E0A93EB807CC
:102E30001CF028E030E00FC00DB407FEF5CF8EB5D2
:102E4000FB01E20FF31F80832F5F3F4F24173507ED
:102E50002CF321E030E0C901DF91CF910895DC012E
:102E600083E480931E0540E050E020E030E019C08C
:102E7000FD01E20FF31F80818EBD09C04F5F5F4FE0
:102E800083E0493E58071CF028E030E00FC00DB445
:102E900007FEF4CF8EB5F901E25EFA4F82832F5F11
:102EA0003F4F2617370724F321E030E020931F051A
:102EB000FB01E05EFA4F1082CB0103960E943B01BA
:102EC0000895BC0184E480931E0540E050E020E0BA
:102ED00030E014C01EBC08C083E0493E580714F01F
:102EE00088E010C04F5F5F4F0DB407FEF5CF8EB581
:102EF000F901E25EFA4F82832F5F3F4F26173707B3
:102F00004CF381E080931F05FB01E05EFA4F1082D5
:102F1000CB0103960E943B01089593E490931E0514
:102F2000282F30E090E008C0E60FF71F80818EBDAB
:102F30000DB407FEFDCF9F5FE92FF0E0E217F30726
:102F40009CF381E080931F051092200583E090E0C0
:102F50000E943B01089581E480931E051CBC1DBCAA
:102F600010927E0310927F031092800381E0809381
:102F70001F051092200583E090E00E943B01089518
:102F800090E490931E050E94621680931F05109294
:102F9000200583E090E00E943B010895CF93DF93EA
:102FA000EC0188818334A9F0843428F4803441F022
:102FB000813401F50BC0843491F08534D9F413C009
:102FC0008A816B814C810E94C0171FC00E94AB1781
:102FD0001CC08A812396BE010E948D1716C08A816B
:102FE00090E00E9461176A81CE01039670E00E9412
:102FF0002F170BC080931E0583E080931F0510924E
:10300000200583E090E00E943B01DF91CF9108957D
:10301000209A219A229A2398249A259A2C982D98BE
:1030200081E08093890382E080938A0380938B03FD
:1030300080938C0381E090E00895109289031092B0
:103040008A0310928B0310928C0381E090E0089524
:10305000289829982A9880E29EE40197F1F7289A07
:103060008AE0982F9A95F1F72A9A299A8A95F1F78A
:103070000895282F299887FD02C02A9801C02A9A0E
:103080008AE0982F9A95F1F7299A8A95F1F729986D
:1030900026FF02C02A9A01C02A988AE0982F9A95A2
:1030A000F1F7299A8A95F1F70895880F20E03AE020
:1030B000299887FF02C02A9A01C02A98932F9A95CF
:1030C000F1F7299A932F9A95F1F72F5F273011F096
:1030D000880FEECF089520E03AE0299887FF02C0DC
:1030E0002A9A01C02A98932F9A95F1F7299A932F3B
:1030F0009A95F1F72F5F283011F0880FEECF0895E1
:1031000029982A988AE0982F9A95F1F7299A982F6A
:103110009A95F1F729982898982F9A95F1F7299A76
:10312000982F9A95F1F729988A95F1F7289A80E0D7
:103130000895299828982A982B9A08950E9428186B
:1031400080E30E94391880E60E94551808950E9475
:10315000281880E00E94391880E00E9455182998AC
:1031600028982A982B9A08950F931F93182F062FAB
:103170000E94281880E40E943918812F0E94551857
:10318000802F0E946B1881E01F910F9108951F936B
:10319000182F0E94281880EC0E943918812F0E9455
:1031A00055180E9480181F91089529988AE08A95E1
:1031B000F1F72A9820E080E04AE0880F299A942FBE
:1031C0009A95F1F729981B998F5F3AE0942F9A9579
:1031D000F1F72F5F283089F72898299A932F9A952D
:1031E000F1F7289A2998932F9A95F1F708951F934C
:1031F000182F0E94281880E80E943918812F0E94F9
:1032000055180E94D5181F910895DF92EF92FF92F2
:103210000F931F93CF93DF93D82E7B018A01C0E0D9
:10322000D0E009C08D2D8C0F0E94F718F801EC0F2B
:10323000FD1F80832196CE15DF05A0F381E090E08D
:10324000DF91CF911F910F91FF90EF90DF90089544
:103250000F931F93182F062F0E949E18812F602F07
:103260000E94B41881E01F910F910895DF92EF92B0
:10327000FF920F931F93CF93DF93D82E7B018A0188
:10328000C0E0D0E009C0F801EC0FFD1F8D2D8C0FC0
:1032900060810E9428192196CE15DF05A0F381E0F8
:1032A00090E0DF91CF911F910F91FF90EF90DF9011
:1032B000089594E090931E050E94361980931F058F
:1032C0001092200583E090E00E943B010895EF9268
:1032D000FF920F931F938B019EE1E92E95E0F92E4B
:1032E00093E090931E05A7014E5F5F4F0E94051962
:1032F00080931F050E5F1F4FE00EF11EF701108235
:10330000C80101960E943B011F910F91FF90EF9021
:10331000089582E080931E051092890310928A031B
:1033200010928B0310928C0381E080931F05109202
:10333000200583E090E00E943B01089581E08093A6
:103340001E050E94081880931F051092200583E037
:1033500090E00E943B010895FC018381823069F076
:10336000833018F48130E1F405C0833049F08430B3
:10337000B9F40EC00E949E1908950E9489190895FB
:103380006581848170E03696AF010E9467190895C7
:103390006581848170E03696AF010E9459190895C5
:1033A000808180931E0583E080931F051092200585
:1033B00083E090E00E943B0108951F920F920FB6A8
:1033C0000F9211240F900FBE0F901F9018959C0123
:1033D0000897029718F024E030E025C0F901E95879
:1033E000FC4F8DE0828328303105A1F02930310572
:1033F00019F027E030E017C0259A81E090E0909323
:1034000089008093880081E88093800089E0809320
:10341000810007C0249A81E08093B30089E68093FD
:10342000B00021E030E0C90108959C01FC01E95899
:10343000FC4F82818D3019F026E030E054C02830F6
:10344000310531F12930310519F027E030E04BC06A
:1034500063307105A9F0643071053CF46130710589
:1034600059F062307105E9F509C06430710551F019
:1034700065307105B1F508C081E007C082E005C084
:1034800083E003C084E001C085E08093810029C00F
:1034900064307105E9F06530710554F462307105EE
:1034A00099F06330710594F461307105D1F40AC06C
:1034B0006630710589F06630710564F0673071051A
:1034C00081F40CC089E60BC08AE609C08BE607C010
:1034D0008CE605C08DE603C08EE601C08FE68093C2
:1034E000B00021E030E0C90108959C01FC01E958D9
:1034F000FC4F82818D3019F026E030E012C0283078
:10350000310559F02930310519F027E030E009C0C4
:10351000709389006093880002C06093B30021E03B
:1035200030E0C90108959C0183E580931E05F901EF
:10353000E958FC4F82818D3019F086E090E012C08E
:103540002830310559F02930310519F087E090E035
:1035500009C0709389006093880002C06093B30033
:1035600081E090E080931F051092200583E090E0B9
:103570000E943B01089522E520931E050E94151A22
:1035800080931F051092200583E090E00E943B018C
:10359000089520E520931E050E94E71980931F05DA
:1035A0001092200583E090E00E943B010895FC0109
:1035B000E958FC4F12828830910531F0893091052D
:1035C00031F026E030E00BC01092B00004C0109241
:1035D0008100109280000E94DE1221E030E0C901DB
:1035E000089521E520931E050E94D71A80931F0598
:1035F0001092200583E090E00E943B010895FC01B9
:103600008081813579F0823518F48035F1F405C078
:10361000823569F08335C9F411C0828190E00E943F
:10362000C91A0895828190E00E94F11A0895638179
:10363000828190E070E00E94BB1A089563818281CC
:1036400090E070E00E94931A089580931E0583E035
:1036500080931F051092200583E090E00E943B01BB
:103660000895DF93CF93CDB7DEB7CF91DF91089563
:103670008A3310F4805301C087556A3310F46053C5
:1036800001C067556F708295807F862B08951F93C8
:10369000682F62956F70182F1F706A3010F4605D8C
:1036A00001C0695A80E00E947A061A3010F4105D59
:1036B00001C0195A80E0612F0E947A061F91089577
:1036C0001F93182F8A3021F480E06DE00E947A0663
:1036D00080E0612F0E947A0681E090E01F910895BA
:1036E00080E00E94AF0508950F9380E00E94950549
:1036F00080E069E140E020E000E00E94D10580E048
:1037000061E00E94E30580E068E00E94020680E03C
:103710006EE40E942E068EEF92E09093B5068093A1
:10372000B4060F9108958230A1F0833028F48823E5
:1037300061F0813039F40BC0843079F0843058F076
:10374000853079F020E030E016C082E107C08EE0DD
:1037500005C088E003C086E001C082E08093E200FB
:1037600002C01092E2008CE08093E30087E3809334
:10377000E40021E030E0C9010895813091F081300A
:1037800038F08230B9F0833019F120E030E031C0F8
:103790008091DB008F778093DB008091DB008F7D51
:1037A00011C08091DB0080688093DB008091DB009A
:1037B0008F7D16C08091DB0080688093DB00809154
:1037C000DB0080628093DB008091DB008F7E0DC088
:1037D0008091DB0080688093DB008091DB00806259
:1037E0008093DB008091DB0080618093DB0021E02F
:1037F00030E0C90108951F93282F162F8FE0809382
:103800008A0380938B031092AD06442319F081E064
:103810008093AD061092A1061092A2061092A30604
:103820001092A406E5EAF6E0119286E0ED3AF80778
:10383000D9F790E0892F8295807F8093ED001092D8
:10384000EE001092EF009F5F9F30A1F7822F0E9441
:10385000931B892B89F0812F0E94BD1B892B61F05E
:103860008091D80082608093D8008091D90082FF37
:10387000FCCF21E030E002C022E030E0C9011F911E
:1038800008958295807F8093ED0008959B01AC019F
:103890008091AD06882381F4822F8295880F807EE7
:1038A0008093F60063E056954795379527956A957E
:1038B000D1F72093F7000895DA01C90153E0880F8A
:1038C000991FAA1FBB1F5A95D1F787608093F400F8
:1038D000292F3A2F4B2F55272093F5009D01442780
:1038E00055272093F6008B2F9927AA27BB27809373
:1038F000F7000895EF92FF920F931F938091AD060A
:103900008823C1F42091F20022952695277030E09B
:1039100040E050E08091F30090E003E0880F991FB1
:103920000A95E1F77C0100E010E0E22AF32A042B7B
:10393000152B33C02091F3008091F200E090F1004C
:103940006091F00090E0A0E0B0E0DC0199278827CA
:1039500030E040E050E0522F442733272227822BCB
:10396000932BA42BB52BFF2400E010E0102F0F2D7C
:10397000FE2CEE248E299F29A02BB12BE62EFF24AE
:1039800000E010E0E82AF92A0A2B1B2B73E01695B9
:103990000795F794E7947A95D1F7B701C8011F917D
:1039A0000F91FF90EF9008959B01AC018091AD06BF
:1039B000882371F4822F8295880F807E8093F20095
:1039C000E3E05695479537952795EA95D1F725C0B9
:1039D00073E0220F331F441F551F7A95D1F7809152
:1039E000F00090E0A0E0B0E087709070A070B07040
:1039F000282B392B4A2B5B2B2093F000BB27A52FBC
:103A0000942F832F8093F100CA01AA27BB278093AC
:103A1000F200252F3327442755272093F3000895DC
:103A2000982F8091AD06882321F08091EF0080616E
:103A300003C08091EF008F7E8093EF00923091F170
:103A4000933028F4992359F0913031F422C0933007
:103A5000B9F1943009F447C020E030E05AC08091B9
:103A6000EF008F7B8093EF008091EF008F77809342
:103A7000EF008091EF008F7D8093EF008091F00048
:103A80008B7F8093F0008091F4008B7F8093F40013
:103A90003EC08091EF008E7F8093EF008091EF0019
:103AA00081601BC08091EF008F778093EF00809141
:103AB000EF0080648093EF008091EF008F7D20C045
:103AC0008091EF008F7B8093EF008091EF00806802
:103AD0008093EF008091EF008F7D8093EF008091C5
:103AE000F0008B7F12C08091EF008F7B8093EF00FE
:103AF0008091EF0080688093EF008091EF008062FA
:103B00008093EF008091F00084608093F00021E0CA
:103B100030E0C9010895FF920F931F93162F042FD1
:103B2000F52E8295807F8093ED0084E00E94101D29
:103B3000193008F018E08091EF00807F812B80938E
:103B4000EF00202F3F2DC901FC0190E004C08191BE
:103B50008093FA009F5F9117D0F31F910F91FF9010
:103B600008959F92AF92BF92CF92DF92EF92FF9211
:103B70000F931F93962E59016A01982F9295907F6B
:103B80009093ED00E82FF0E0883080F42091DE0083
:103B9000E45FFC4F81E090E0008002C0880F991F35
:103BA0000A94E2F7282B2093DE000FC02091DF005B
:103BB000E45FFC4F81E090E0008002C0880F991F15
:103BC0000A94E2F7282B2093DF00C801B7010E9476
:103BD000461CC601B5010E94D41C892D0E94101DEF
:103BE000892B19F021E030E002C022E030E0C90169
:103BF0001F910F91FF90EF90DF90CF90BF90AF900B
:103C00009F9008958091EF0087FD04C08091EF00A0
:103C100086FF3CC08091EF0087FD0AC08091EF00D5
:103C200086FF06C08091F00082FD02C081E0089509
:103C30008091EF0087FD0AC08091EF0086FF06C0EB
:103C40008091F00082FF02C082E008958091EF0031
:103C500087FF0AC08091EF0086FD06C08091F000CA
:103C600082FD02C083E008958091EF0087FF0EC0BF
:103C70008091EF0086FD0AC08091EF0085FF06C0AD
:103C80008091F00082FF02C084E0089580E00895F2
:103C9000EF92FF920F931F93162F042FF52E82950C
:103CA000807F8093ED000E94021EE82E193008F0FC
:103CB00018E08091EF00807F812B8093EF00202F10
:103CC0003F2DC901FC0190E004C081918093FA006E
:103CD0009F5F9117D0F381E00E94101D8091EE004C
:103CE00086FFFCCF8091EE008F7B8093EE008E2DBF
:103CF0000E94101D81E090E01F910F91FF90EF90C6
:103D00000895482F893008F048E08091EF00807FC7
:103D1000842B8093EF00FB0190E004C0819180939D
:103D2000FA009F5F9417D0F30895AC0120E030E0D3
:103D30008091FA00FA01E20FF31F80832F5F3F4F5B
:103D400028303105A9F70895E82FF0E0883080F495
:103D50002091DE00E45FFC4F81E090E0008002C033
:103D6000880F991F0A94E2F7282B2093DE0008950C
:103D70002091DF00E45FFC4F81E090E0008002C012
:103D8000880F991F0A94E2F7282B2093DF000895EB
:103D9000AEEDB0E02C91ECE0F3E0E80FF11D81E036
:103DA00090E0008002C0880F991F0A94E2F7809586
:103DB00082238C9308953091E0002091E100922FAE
:103DC00080E0232F30E0282B392B2115310521F4F9
:103DD00007C0369527958F5F20FFFBCF8F3008F007
:103DE0008FEF0895982F9295907F9093ED00AEED10
:103DF000B0E02C91ECE0F3E0E80FF11D81E090E001
:103E0000008002C0880F991F0A94E2F780958223F0
:103E10008C9380E00E94101D81E090E008951F9334
:103E200010928A0310928B0310E0812F0E94F21EE1
:103E30001F5F1F30D1F78091D8008D7F8093D8000D
:103E40008091D90082FDFCCF81E090E01F91089520
:103E50001F938295807F8093ED000E94021E182F91
:103E600082E00E94101D8091EE0086FFFCCF8091C1
:103E7000EE008F7B8093EE00812F0E94101D81E069
:103E800090E01F9108951F920F920FB60F920BB6FC
:103E90000F9211241F932F933F934F935F936F9330
:103EA0007F938F939F93AF93BF93EF93FF93109163
:103EB000ED003091E0002091E100922F80E0232F6F
:103EC00030E0282B392B21153105A9F103C0369597
:103ED00027958F5F20FFFBCF8F3068F58F3F59F11B
:103EE0008295807F8093ED000E947A1C6093A106EA
:103EF0007093A2068093A3069093A406E5EAF6E0E9
:103F00008091FA00819386E0ED3AF807C9F70E94A4
:103F10007A1C6093A1067093A2068093A3069093E7
:103F2000A4068091EE008F7D8093EE0083E00E94D6
:103F3000101D1093ED00FF91EF91BF91AF919F91F4
:103F40008F917F916F915F914F913F912F911F9131
:103F50000F900BBE0F900FBE0F901F90189586E725
:103F600080931E0581E080931F058091A1069091AA
:103F7000A206A091A306B091A40680932005292F44
:103F80003A2F4B2F5527209321059D014427552774
:103F9000209322058B2F9927AA27BB2780932305DF
:103FA0001092A1061092A2061092A3061092A406E7
:103FB000A5EAB6E026E030E08C91F901E25EFA4F26
:103FC00080831D922F5F3F4F86E0AD3AB807A1F77F
:103FD00010922C058FE090E00E943B01089595E738
:103FE00090931E050E94281F80931F0510922005A4
:103FF00083E090E00E943B01089594E790931E05B2
:104000000E94F21E80931F051092200583E090E02D
:104010000E943B01089592E790931E050E94481E5E
:1040200080931F051092200583E090E00E943B01E1
:104030000895EF92FF920F931F9393E790931E05BD
:104040000E94B11D80931F051092200583E090E02F
:104050000E943B011F910F91FF90EF9008950E94E5
:104060008B1D87E780931E0581E080931F051092CA
:10407000200583E090E00E943B01089581E7809352
:104080001E050E940F1F80931F051092200583E0DC
:1040900090E00E943B010895462F90E790931E0503
:1040A00062E00E94FB1B80931F051092200583E0B5
:1040B00090E00E943B010895EF92FF920F931F93AF
:1040C000FC018081833701F1843748F48137C9F0DE
:1040D000823708F06BC0803709F07FC00DC085378C
:1040E00009F46BC0853708F45DC0863709F469C0F0
:1040F000873709F072C06AC0828163810E944C20B8
:1041000077C00E943E2074C00000258130E040E06E
:1041100050E0542F432F322F2227868190E0A0E0D9
:10412000B0E0DC0199278827280F391F4A1F5B1F41
:104130008481280F311D411D511D878190E0A0E031
:10414000B0E0B82FAA2799278827280F391F4A1FC0
:104150005B1FE184FF2400E010E0102F0F2DFE2CE8
:10416000EE24828590E0A0E0B0E0DC01992788276A
:10417000E80EF91E0A1F1B1F8085E80EF11C011DA9
:10418000111D838590E0A0E0B0E0B82FAA27992701
:104190008827E80EF91E0A1F1B1F828163810E9477
:1041A000192026C082810E94FD1F22C08281638166
:1041B0003496AF010E940B201BC082810E94EF1F2A
:1041C00017C0828190E00E94AF1F12C0828163817C
:1041D0003496AF010E942F200BC080931E0583E010
:1041E00080931F051092200583E090E00E943B0120
:1041F0001F910F91FF90EF900895DC0180E1A030B6
:10420000B80710F082E00895F999FECF9D010BC028
:10421000F999FECF32BD21BDF89A80B5E60FF71FA0
:1042200080832F5F3F4F822F8A1BE82FF0E0E41737
:10423000F50770F381E00895DC0180E1A030B80754
:1042400010F082E00895F999FECF9D0110C0E60FAD
:10425000F71FE081F999FECFC901019632BD21BD5A
:10426000E0BD0FB6F894FA9AF99A0FBE9C01822F1E
:104270008A1BE82FF0E0E417F50748F3C9010E9414
:10428000FD2081E008950F931F938B0121E8209377
:104290001E050E941C2180931F051092200500D04E
:1042A00000D000D0EDB7FEB731968BE193E0ADB70B
:1042B000BEB712969C938E93119783E293E09383FB
:1042C00082838AE590E0958384830E940D250F9078
:1042D0000F908CE293E0EDB7FEB792838183148355
:1042E00003830E940D250F900F900F900F9083E095
:1042F00090E00E943B011F910F910895CF92DF92B1
:10430000EF92FF920F931F937B010EE115E020E8DF
:1043100020931E0522E0C22ED12CC00ED11EB60164
:10432000A7010E94FD2080931F0582E090E0E80E27
:10433000F91E0E0D1F1DD8011C9200D000D000D018
:10434000EDB7FEB731968BE193E0ADB7BEB71296ED
:104350009C938E93119783E293E09383828385E30A
:1043600090E0958384830E940D250F900F9089E340
:1043700093E0EDB7FEB792838183D482C3820E941B
:104380000D250F900F900F900F90C70101960E947E
:104390003B011F910F91FF90EF90DF90CF90089518
:1043A000EF92FF920F931F93CF93DF93EC019B81CA
:1043B00080E02A817C01E20EF11C9D8180E02C814D
:1043C0008C01020F111D00D000D000D0EDB7FEB758
:1043D00031968BE193E0ADB7BEB712969C938E9366
:1043E000119783E293E0938382838AE190E095833F
:1043F00084830E940D25EDB7FEB7319683E493E0E8
:10440000ADB7BEB712969C938E9311971383028318
:10441000F582E4820E940D2588812DB73EB72A5F80
:104420003F4F0FB6F8943EBF0FBE2DBF803819F036
:10443000813869F405C0C701B8010E947E2112C00D
:104440002696C701BE01A8010E9443210BC080939C
:104450001E0583E080931F051092200583E090E005
:104460000E943B01DF91CF911F910F91FF90EF9040
:104470000895CF93DF93EB0190E003978632910587
:1044800048F4865B9F4FFC01EE0FFF1F0590F491EF
:10449000E02D099480E0BCC188E290E09983888394
:1044A00086E290E09B838A8387E290E0B0C088E256
:1044B00090E09983888386E290E09B838A8387E2F9
:1044C00090E058C188E290E09983888386E290E08A
:1044D0009B838A8387E290E076C088E290E09983AC
:1044E000888386E290E09B838A8387E290E05DC0C8
:1044F00088E290E09983888386E290E09B838A83B8
:1045000087E290E044C088E290E09983888386E265
:1045100090E09B838A8387E290E02BC088E290E062
:104520009983888386E290E09B838A8387E290E088
:104530005CC181E390E0998388838FE290E09B8364
:104540008A8380E390E05FC181E390E09983888370
:104550008FE290E09B838A8380E390E046C181E311
:1045600090E0998388838FE290E09B838A8380E345
:1045700090E09D838C8385E049C181E390E099833D
:1045800088838FE290E09B838A8380E390E09D8321
:104590008C8384E03BC181E390E0998388838FE240
:1045A00090E09B838A8380E390E09D838C8383E00B
:1045B0002DC181E390E0998388838FE290E09B8313
:1045C0008A8380E390E09D838C8382E01FC181E336
:1045D00090E0998388838FE290E09B838A8380E3D5
:1045E00090E0C8C081E390E0998388838FE290E0F7
:1045F0009B838A8380E390E00AC08EE290E09983F7
:1046000088838CE290E09B838A838DE290E09D8397
:104610008C831E82FCC08EE290E0998388838CE2BA
:1046200090E09B838A838DE290E0A4C08EE290E0CC
:10463000998388838CE290E09B838A838DE290E06B
:10464000C2CF8EE290E0998388838CE290E09B83D6
:104650008A838DE290E0A9CF8EE290E099838883EF
:104660008CE290E09B838A838DE290E082CF8EE2A1
:1046700090E0998388838CE290E09B838A838DE22B
:1046800090E0B3C08EE290E0998388838CE290E062
:104690009B838A838DE290E0B6C085E290E09983A7
:1046A000888383E290E09B838A8384E290E0AFCFAB
:1046B00085E290E09983888383E290E09B838A83FC
:1046C00084E290E057C085E290E09983888383E29A
:1046D00090E09B838A8384E290E075CF85E290E04E
:1046E0009983888383E290E09B838A8384E290E0CD
:1046F0005CCF85E290E09983888383E290E09B839E
:104700008A8384E290E043CF85E290E099838883B6
:1047100083E290E09B838A8384E290E02ACF85E263
:1047200090E09983888383E290E09B838A8384E28C
:1047300090E05BC085E290E09983888383E290E01B
:104740009B838A8384E290E05EC08BE290E0998351
:10475000888389E290E09B838A838AE290E057CF46
:104760008BE290E09983888389E290E09B838A833F
:104770008AE290E09D838C8381E08E8349C08BE246
:1047800090E09983888389E290E09B838A838AE220
:1047900090E019CF8BE290E09983888389E290E0E2
:1047A0009B838A838AE290E000CF8BE290E099833A
:1047B000888389E290E09B838A838AE290E0E7CE57
:1047C0008BE290E09983888389E290E09B838A83DF
:1047D0008AE290E0CECE8BE290E09983888389E2F2
:1047E00090E09B838A838AE290E09D838C8386E0BD
:1047F0000DC08BE290E09983888389E290E09B83EF
:104800008A838AE290E09D838C8387E08E8381E0B7
:10481000DF91CF910895CF93DF93BC018230910552
:1048200010F462E070E0A091B006B091B106ED0125
:10483000E0E0F0E040E050E021C0888199818617F7
:10484000970769F48A819B81309719F0938382835B
:1048500004C09093B1068093B006FE0134C068177F
:10486000790738F44115510519F08417950708F4B4
:10487000AC01FE018A819B819C01E9012097E9F648
:1048800041155105A9F1CA01861B970B049708F43D
:10489000BA01E0E0F0E02AC08D919C911197841755
:1048A0009507F9F46417750781F412968D919C9120
:1048B0001397309719F09383828304C09093B106C5
:1048C0008093B006FD0132964CC0CA01861B970B3F
:1048D000FD01E80FF91F6193719302978D939C93EB
:1048E00040C0FD01828193819C01D9011097A1F6FE
:1048F0008091AE069091AF06892B41F480916A03B6
:1049000090916B039093AF068093AE0640916C0339
:1049100050916D034115510541F44DB75EB780913B
:10492000680390916903481B590B2091AE063091A2
:10493000AF06CA01821B930B8617970780F0AB0165
:104940004E5F5F4F8417950750F0420F531F5093EF
:10495000AF064093AE06F9016193719302C0E0E0A7
:10496000F0E0CF01DF91CF910895CF93DF930097CF
:1049700009F450C0EC0122971B821A82A091B00664
:10498000B091B106109709F140E050E0AC17BD07B7
:1049900008F1BB83AA83FE0121913191E20FF31F3D
:1049A000AE17BF0779F48D919C911197280F391F8D
:1049B0002E5F3F4F3983288312968D919C911397D8
:1049C0009B838A834115510571F4D093B106C0933E
:1049D000B00620C012968D919C911397AD0100975F
:1049E00011F0DC01D3CFFA01D383C283219131913D
:1049F000E20FF31FCE17DF0769F488819981280F32
:104A0000391F2E5F3F4FFA01318320838A819B81BA
:104A100093838283DF91CF910895A0E0B0E0E3E13A
:104A2000F5E20C940B28FE0135966191719180910D
:104A3000B4069091B506AF010E9457252096E2E09A
:104A40000C9427280F931F93CF93DF938C01E09151
:104A5000B406F091B506838181FF21C0C0E0D0E0AB
:104A60000DC0E091B406F091B50620853185BF01F7
:104A7000F9010995892B11F0CFEFDFEFF801819152
:104A80008F01882371F7E091B406F091B506208577
:104A900031858AE0BF01F9010995892B11F0CFEF2B
:104AA000DFEFCE01DF91CF911F910F910895ABE021
:104AB000B0E0EDE5F5E20C94FB273C012B015A0137
:104AC000FC0117821682838181FD03C06FEF7FEFA7
:104AD000C6C19AE0892E1E010894211C311CF301E5
:104AE0002381F20123FD859123FF81912F018823EA
:104AF00009F4B2C1853239F423FD859123FF8191F8
:104B00002F01853229F490E0B3010E944A27E7CFB4
:104B1000982FFF24EE249924FFE1FF15D0F09B325B
:104B200069F09C3228F4903259F0933291F40EC01F
:104B30009D3249F0903369F441E024C052E0F52AF7
:104B400084E0F82A28C098E0F92A25C0E0E1FE2A8E
:104B500022C0F7FC29C0892F80538A3070F4F6FEFA
:104B600005C0989C902C1124980E15C0E89CE02C50
:104B70001124E80EF0E2FF2A0EC09E3229F4F6FC62
:104B80006BC140E4F42A07C09C3619F450E8F52ABA
:104B900002C0983649F4F20123FD959123FF9191CB
:104BA0002F01992309F0B8CF892F8554833018F04D
:104BB0008052833038F444E050E0A40EB51E5FE329
:104BC00059830FC0933631F0933779F0933509F05C
:104BD00056C020C0F5018081898342E050E0A40ED8
:104BE000B51E610101E010E012C0F501C080D18066
:104BF000F6FC03C06FEF7FEF02C0692D70E042E06A
:104C000050E0A40EB51EC6010E943F278C015FE74D
:104C1000F52214C0F501C080D180F6FC03C06FEF0F
:104C20007FEF02C0692D70E042E050E0A40EB51E97
:104C3000C6010E9434278C0150E8F52AF3FE07C014
:104C40001AC080E290E0B3010E944A27EA948E2DB8
:104C500090E008171907A8F30EC0F601F7FC85913C
:104C6000F7FE81916F0190E0B3010E944A27E110A5
:104C7000EA94015010400115110579F7EAC0943605
:104C800011F0993669F5F7FE08C0F50120813181F0
:104C90004281538184E090E00AC0F50180819181D6
:104CA0009C01442737FD4095542F82E090E0A80EE8
:104CB000B91E9FE6F92257FF09C0509540953095DF
:104CC00021953F4F4F4F5F4FE0E8FE2ACA01B901DF
:104CD000A1012AE030E00E947627D82ED21840C0E9
:104CE000953729F41F2D1F7E2AE030E01DC01F2DAF
:104CF000197F9F3661F0903720F4983509F0ACC0E9
:104D00000FC0903739F0983709F0A6C004C028E0EA
:104D100030E00AC0106114FD146020E130E004C0EE
:104D200014FD166020E132E017FF08C0F501608134
:104D300071818281938144E050E008C0F501808157
:104D40009181BC0180E090E042E050E0A40EB51EED
:104D5000A1010E947627D82ED2188FE7F82EF122D3
:104D6000F6FE0BC05EEFF522D91438F4F4FE07C04E
:104D7000F2FC05C08FEEF82202C01D2D01C0192DD6
:104D8000F4FE0DC0FE01ED0DF11D8081803319F49C
:104D900099EEF92208C01F5FF2FE05C003C08F2DF7
:104DA000867809F01F5F0F2DF3FC14C0F0FE0FC0D2
:104DB0001E1510F09D2C0BC09D2C9E0C911A1E2DC3
:104DC00006C080E290E0B3010E944A271F5F1E15D3
:104DD000C0F304C01E1510F4E11A01C0EE2404FF54
:104DE0000FC080E390E0B3010E944A2702FF1DC07C
:104DF00001FD03C088E790E00EC088E590E00BC09D
:104E0000802F867891F001FF02C08BE201C080E222
:104E1000F7FC8DE290E0B3010E944A2706C080E3D0
:104E200090E0B3010E944A279A94D914C0F3DA940F
:104E3000F101ED0DF11D808190E0B3010E944A2740
:104E4000DD20A9F706C080E290E0B3010E944A2766
:104E5000EA94EE20C1F743CEF30166817781CB015E
:104E60002B96E2E10C941728FC01059061507040EC
:104E70000110D8F7809590958E0F9F1F0895FC0123
:104E80006150704001900110D8F7809590958E0F79
:104E90009F1F08950F931F93CF93DF938C01EB0116
:104EA0008B8181FF1BC082FF0DC02E813F818C81D1
:104EB0009D812817390764F4E881F9810193F9830A
:104EC000E88306C0E885F985802F0995892B31F4A0
:104ED0008E819F8101969F838E8302C00FEF1FEF0B
:104EE000C801DF91CF911F910F910895FA01AA2770
:104EF000283051F1203181F1E8946F936E7F6E5F1D
:104F00007F4F8F4F9F4FAF4FB1E03ED0B4E03CD0CA
:104F1000670F781F891F9A1FA11D680F791F8A1FAD
:104F2000911DA11D6A0F711D811D911DA11D20D014
:104F300009F468943F912AE0269F11243019305DCE
:104F40003193DEF6CF010895462F4770405D4193BF
:104F5000B3E00FD0C9F7F6CF462F4F70405D4A330C
:104F600018F0495D31FD4052419302D0A9F7EACFD4
:104F7000B4E0A6959795879577956795BA95C9F703
:104F800000976105710508959B01AC010A2E0694F6
:104F90005795479537952795BA95C9F7620F731FAF
:104FA000841F951FA01D089597FB092E07260AD080
:104FB00077FD04D00CD006D000201AF470956195CE
:104FC0007F4F0895F6F7909581959F4F0895AA1BFE
:104FD000BB1B51E107C0AA1FBB1FA617B70710F0E4
:104FE000A61BB70B881F991F5A95A9F78095909516
:104FF000BC01CD0108952F923F924F925F926F9224
:105000007F928F929F92AF92BF92CF92DF92EF9258
:10501000FF920F931F93CF93DF93CDB7DEB7CA1BD9
:10502000DB0B0FB6F894DEBF0FBECDBF09942A8804
:10503000398848885F846E847D848C849B84AA84AC
:10504000B984C884DF80EE80FD800C811B81AA8139
:10505000B981CE0FD11D0FB6F894DEBF0FBECDBF04
:08506000ED010895F894FFCF63
:10506800456D62656464656450726F6A65637473E4
:10507800004F63746F70757355534220496E7465A1
:10508800726661636520436F6E766572746572201F
:10509800616E6420492F4F20457874656E73696F7F
:1050A8006E0032303039303731380025732C2564A2
:1050B8003A20006D61696E2E630066697273742010
:1050C8007061636B6574206F662061206C6F6E671A
:1050D800206D65737361676520286C656E677468F9
:1050E8003A202564290A006F63746F707573206C09
:1050F8006F6E672072756E6E696E67206D6573736B
:10510800616765006F63746F7075732E6C6F6E677F
:105118005F696E646578203C206F63746F70757387
:105128002E6C6F6E675F6279746573006E6F7420A2
:105138006C617374207061636B65743A206469668E
:1051480066203E203634006C617374207061636B96
:105158006574007061727365722C20636865636B97
:105168003A2025582C20636F6D6D616E643A2025B6
:10517800580A0063616C6C696E6720696F5F7061C3
:10518800727365720063616C6C696E672061646339
:105198005F7061727365720063616C6C696E672021
:1051A8006932635F7061727365720063616C6C6908
:1051B8006E67207370695F706172736572006361F6
:1051C8006C6C696E672070776D5F70617273657261
:1051D8000063616C6C696E672063616E5F706172F9
:1051E8007365720063616C6C696E672065657072C7
:1051F8006F6D5F70617273657200756E6B6E6F773D
:105208006E20636D6400726563656976696E6720F8
:10521800636F6D6D616E643A20255820286C656E49
:105228006774683A202575290A00676574206E65D9
:1052380078740067657420616E64206578656375AD
:1052480074650009040025732C25643A2000616404
:10525800632E6300576572742025690D0A000000EB
:10526800000200000000601B0000000000010203B3
:10527800040506070001020304050625732C2564AE
:105288003A2000656570726F6D2E630077726974DD
:1052980074656E3A2025730A00726561643A2025A8
:1052A800730A00656570726F6D5F70617273657205
:1052B8003A206C656E6774683A2025752C20616405
:0E52C80064723A2025750A002000B806000026
:00000001FF
